:030000000219FDE5
:03000B000200AA46
:03002B0002015778
:03005B000202E6B8
:030073000202D3B3
:1000800002030406080C10182030406080040608A3
:100090000C10182030406080A0C00003070F1F0D17
:1000A0000D04050D050205030302C2AFC0D0C0E078
:1000B000206214E5256009E473E525F4F58AD2622F
:1000C000D0E0D0D0D2AF3285268AC262E526F46075
:1000D0002AD0E0D0D0C295C294C293D2AF32C2959A
:1000E000C294C293206F0D20650A7405D5E0FDE52A
:1000F0007BF45290D0E0D0D0D2AF32758A00C28D5E
:10010000D26201F401B9306805206502D29501B9C7
:10011000306805206502D29401B930680520650277
:10012000D29301B9D29230680A2065077403D5E0F2
:10013000FDD29501B9D29130680A2065077403D5C4
:10014000E0FDD29401B9D29030680A2065077403AB
:10015000D5E0FDD29301B9C2AFC2AD53E6EFC0D036
:10016000C0E0D2D3D2AFC2CEE52A600720744F15CB
:100170002A21BE7800790020742EE580307E01F4BB
:1001800030E70278FF53DACF207E0343DA20307E57
:100190000343DA10C2D8C271E580307E01F430E743
:1001A0000279FFC3E89970CB306103752A18207477
:1001B00003752A18885CD270E86003755F002074AC
:1001C0000DE52B6004152B21CE43DA01C2D8207037
:1001D00002413DA85C206102C2702074367982B76A
:1001E0000431C3E894F0400374F0F8E8C4540F28D5
:1001F000F87984B703024113C313C313872120087E
:1002000002C313200A06C3C898F8411328F8500304
:1002100074FFF88822E52D54066022206B1FE53616
:10022000C333C333F8E564C313C313F9C395224042
:10023000028922E82522F52250037522FF7882B632
:10024000044E852224A824C3E52495614002A861B8
:10025000C3E895634002A8638825E5667002418E75
:10026000C3E8AA669A5003E8FAE4F9EAC333FBE567
:1002700068F45B29400D2567F8E567600215674063
:100280000B418E0AC3E5679A5002056778FF8826FE
:1002900020CF0AD0E0D0D043E610D2AD32C2CF0595
:1002A0003A7801E52A6005307402152AC3E55C94AA
:1002B000014005755F0041C9756000756900E55F23
:1002C0002401F55F5003755FFFD0E0D0D043E61006
:1002D000D2AD32C2AF53E67F7592FA7593FFC2601A
:1002E000759104D2AF32C2AF53E6EFC2ADC0D0C0F9
:1002F000E0C0F0D2D3D2AFA8FBA9FCC2D8307102C3
:10030000614D53DACF207E0343DA10307E0343DAA7
:1003100020D271E580307E01F420E7026124882735
:100320008928A17A53DACF207E0343DA20307E0376
:1003300043DA10C2D8C271307402A1667800E58039
:10034000307E01F430E702A166885CA14E53DACF1B
:10035000207E0343DA20307E0343DA10C27120612D
:1003600002812653DACF207E0343DA10307E034326
:10037000DA20C2D8D27188578958C3E89555F8E970
:100380009556F97B007E087A00C3E8948CE99400C6
:100390005005755B008118882178A2E6A821605578
:1003A000C3E894C8E994005008E4D2E4FB7A0A61F7
:1003B000F3C3E89468E994015008E4D2E3FB7A0FB0
:1003C00061F3C3E894D0E994025008E4D2E2FB7AE6
:1003D0001E61F3C3E894A0E994055008E4D2E1FB60
:1003E0007A3C61F3C3E89498E994085008E4D2E0B9
:1003F000FB7A787E00C3E89559FCE9955AFD30E711
:100400000AECF42401FCEDF43400FD755B00C3EC50
:100410009AED9E5003755B018859895A8557558519
:1004200058567802A14EC3E89527F8E99528F93087
:100430007C02A132307B02A132307A02A12B2075DE
:10044000028149E9FDE8FC8168E9C313F9E813F882
:10045000307902A12BE9C313F9E813F8307802A12F
:100460002BE9C313FDE813FC20612CC3EC941CEDB5
:0F04700094024002817FED701EC3EC94C85018B7
:10047F000529E52970021529C3E529940A5002A11F
:10048F0066755C00D270A166E5296002152978882F
:10049F00E6F97400207F087896B90302789EE62467
:1004AF00FAFEE43400FFC3EC9EFCED9FFD9208B909
:1004BF000310A2085007207609D27681D130760238
:1004CF00C276A2085016B9030DECF42401FCEDF42A
:1004DF003400FD0204EB78007900A132B90315EC6A
:1004EF0033FCED33FDC3EC940AFCED9400FD500496
:1004FF007C007D00C3EC94FFED9400400678FF79FB
:10050F0000A132EC8572F0A4C5F0A2F733F87900A0
:10051F00400302054E78FF790002054EE9C313F937
:10052F00E813F8307C0EE9600278FFC3E81338F85F
:10053F00E43400F9C3E894FFE99400400278FF889F
:10054F005CD270206102A166741FF4552F4BF52FFA
:10055F00C274EB7002D274752A18307403752A0AAC
:10056F00306102A17A20740353DAFE207403752BD5
:10057F0006D0F0D0E0D0D0D2AD43E61032790102F0
:10058F0005AA79030205AA790A0205AA791E0205AE
:10059F00AA79640205AA79C80205AA7817E4D5E0FA
:1005AF00FDD8FAD9F6227A147B780205D17A107B1E
:1005BF008C0205D17A0D7BB40205D17A0B7BC80270
:1005CF0005D1E573D5E001227902E4D291D5E0FDA2
:1005DF00D294D5E0FDC294D5E0FDC291D5E0FDE9FE
:1005EF0020E002D29530E002D293E573D5E0FDE929
:1005FF0020E002C29530E002C2937496D5E0FDD997
:10060F00C9EAF8D5E0FDD8FBDBB8D29122C37C0054
:10061F007D0075F00005F0EA33FAEB33FB50F6EB93
:10062F0013FBEA13FAC3E9FFE8FEE89AF8E99BF92E
:10063F005004EFF9EEF8B3EC33FCED33FDD5F0DFFA
:10064F00EDF9ECF822E889F08A20D2D4F8A9F07BF2
:10065F000030F70B7BFFF42401F8E9F43400F9E8DC
:10066F008520F0A4ADF0F8E98520F0A4AFF0FEED01
:10067F002EF974003FFA7C04C3EA13FAE913F9E880
:10068F0013F8DCF48BF030F70AE8F42401F8E9F4FE
:10069F003400F9E889F0C2D4F8A9F0227882B604C0
:1006AF0003020706C3E55C940140030206D08522CE
:1006BF0024E4F544F545F546F547F548C26E0207C3
:1006CF00067882E6FCD26EE522F523783879C7AA40
:1006DF0040AB41C3EB13FBEA13FAEC146013C3EB0B
:1006EF0013FBEA13FAEC14146007C3EB13FBEA13C2
:1006FF00FAD11C8844894522C3E5449523F8E54582
:10070F009400F9500CC3E89480E994FF4016020757
:10071F0037C3E8947FE994005003020737787F7955
:10072F0000020737788079FF8849894A22E54925F1
:10073F0046F8E54A3547F9854A20E4300701F43594
:10074F0048FA30E709C3EA94F04015020775C3EA87
:10075F00940F500302077578FF79FF7A0F02077520
:10076F00780079007AF0C3E5249561500AC37401CB
:10077F009524500B020793E54A20E70E020793E5F5
:10078F004A30E706884689478A482278A5E6FAC3A1
:10079F00E54933F8E54A33F9D154E930E70BC3E8BB
:1007AF009480E994FF4013E1CDC3E8947FE994006E
:1007BF005002E1CD787F7900E1CD788079FFE82094
:1007CF00E715C3E52398F84009C3E89401400302F5
:1007DF0007F478010207F4E8F424012523F8400315
:1007EF000207F478FF884B2278A6E6FAA847A948B3
:1007FF00120654E930E70CC3E89401E994FF401660
:10080F00020829C3E894FFE99400500302082978ED
:10081F00FF7900020829780179FFE920E715C3E580
:10082F004B98F84009C3E89401400302085078013F
:10083F00020850E8F42401254BF8400302085078D1
:10084F00FF88242278FF20692879A1E76023E541FA
:10085F00601F74FF8541F0848539F0306A0375F0AD
:0F086F0005A4F8C5F0600278FFC3E89564500255
:10087E00A864886322C3E5409440E5419401E56392
:10088E005003140194046002F5632202089C227541
:10089E00E890227883E6FF30EDF9A8BDA9BE057079
:1008AE00C3E57094084052757000E9FA79A0E760CC
:1008BE0044EA7007E571601B0208D5C3E8957160C4
:1008CE0010E5715006600C140208E10460F902088C
:1008DE00E1E571F571C3946D401B7561C0C394045D
:1008EE004013756180C39404400B756140C394043A
:1008FE00400375610075BB0622E561241050027439
:10090E00FFF5617982B70402212EC3A861E5249810
:10091E005002A824C3E895634002A8638825882660
:10092E00E570B4070375BB1022743279A787F0A463
:10093E00C5F0A2F733F8C3E895614002A86188229A
:10094E008824882588268864227540007541F02207
:10095E00C2AF75C820A8CCA9CDAA3A30CF010A756E
:10096E00C824D2AFAB3BAC3C883B893CC3E89BF878
:10097E00E99C206908F9306602416F21C9AD3D8AB4
:10098E003DF9EA9DFA600678FF79FF21AEAE3EAFE3
:10099E003F8B3E8C3FA83BA93CC3E89EF8E99FF9EC
:1009AE00C3E54113FBE54013FAE82AF540E93BF5B0
:1009BE004150067540FF7541FF4116AA40AB41AC50
:1009CE0040AD417E047F02C3EB9404400D1E1FC355
:1009DE00EB94084005206A021E1FC3ED13FDEC13B5
:1009EE00FCDEF7C3EA9CFAEB9DFBEF6009C3E9134B
:1009FE00F9E813F8DFF7EA28FAEB39FB8A408B4166
:100A0E0050067BFF8B408B41C3EB94025002D266A3
:100A1E003069047F0341417892E6FFC3E537948243
:100A2E0040110FC3E53794A040010FC3EF94064069
:100A3E00027F057E02E541C4540FF9E541C454F02E
:100A4E00F8E540C4540F28F8C3E89EFAE99400FB79
:100A5E004009C3EA9402EB940050047A02E4FB418D
:100A6E00BBAA40AB41EBC4FEEAC4540F4EFCC3EA32
:100A7E009CFAEB9400FBC3E813C313F8EA28FAEBD5
:100A8E003400FB8A408B41C3EB94024002C266786D
:100A9E0002EBC4FE7B00EAC4540F4EFAC3EA98FA86
:100AAE004005C3940250027A027892E6FF3060024B
:100ABE0041BB855192855293D26043E680C3E49A3E
:100ACE00F8E49BF93066026147E8FAE9FBD3E913D3
:100ADE00FDE813FC88518952C3EF94036038EF2070
:100AEE00E00DE82CF8E93DF9ECFAEDFB020B10E80D
:100AFE0028F8E939F9C3E82402F8E93400F97AFE56
:100B0E007BFFC3EF9403400E8A538B54884D894E5E
:100B1E008C4F8D50617B885389548A4D8B4E8C4FF0
:100B2E008D503069127553F07554FF754FF0755036
:100B3E00FF7551F07552FF617BE8FAD3E813FC881C
:100B4E0051C3EF94036020EF20E007E82CF8ECFA95
:100B5E006167E8282402F87AFEC3EF940340088AFE
:100B6E0053884D8C4F617B88538A4D8C4FE568C3FB
:100B7E00335002646BF5683060026185753402D2C1
:100B8E006043E680E52D54066034A840A941C3E9D0
:100B9E0013F9E813F8C3E913F9E813F8306904E917
:100BAE002440F9C2AF53E67F759100C3E498F594E3
:100BBE00E499F595759104D26043E680D2AF22D2C6
:100BCE0064754300752000306C03752040020BECF9
:100BDE00D264754300752040306C03752000780197
:100BEE007901206620E52D54066002C2647914E571
:100BFE0041C313700104F8C3941440027814306991
:100C0E0004781B791B206010E543600C306903D516
:100C1E003404D26D8196718D0543E59B5440B52009
:100C2E0002818030690908C3E899400118811320B8
:100C3E00640A08C3E899400261EC8113C264C2AF32
:100C4E0053E67F7591003066127594007595F875B0
:100C5E009104D26043E680D2AF61ECE5417EFFC3E2
:0E0C6E00334005C3334001FEC3E49E7594007D
:100C7C00F595815DC3E5339401500261EC3064025B
:100C8C0061ECD80281948113C26DC2AF53E67F75BB
:100C9C009100855394855495759104854D92854E9C
:100CAC0093D26043E680D2AFE52D54066008206AEB
:100CBC00020533020CD2306D0D206C0A206407152E
:100CCC008115810215852278003064027801E537A0
:100CDC0075F007A4F9E5F028F5F0E9A2F013A2F1FC
:100CEC0013A2F213F537C394785003753778C3E524
:100CFC003795384008D265C295C294C293306002D1
:100D0C00A109854F92855093D26043E68022207DC5
:100D1C0016C2AF754202D291C292306202D293D205
:100D2C00AF759F11020F0AC2AF754202D291C290E9
:100D3C00306202D295D2AF759F11020F0A30724306
:100D4C00207D20C2AF754203900135757B02C293A2
:100D5C00D290306204D294A167C291D2AF759F0138
:100D6C00020F0AC2AF754203900135757B02C29522
:100D7C00D292306204D294A187C291D2AF759F21D6
:100D8C00020F0A207D17C2AF754203900110C29367
:100D9C00306202D294D2AF759F01020F0AC2AF75B6
:100DAC004203900110C295306202D294D2AF759F6B
:100DBC0021020F0A207D16C2AF754204D292C29056
:100DCC00306202D294D2AF759F21020F0AC2AF7566
:100DDC004204D290C292306202D294D2AF759F017B
:100DEC00020F0A307243207D20C2AF75420590017C
:100DFC0024757B04C294D291306204D295C10DC289
:100E0C0092D2AF759F11020F0AC2AF7542059001C5
:100E1C0046757B01C294D291306204D293C12DC22B
:100E2C0090D2AF759F11020F0A207D17C2AF754289
:100E3C0005900106C294306202D295D2AF759F1113
:100E4C00020F0AC2AF75420590011AC2943062EBD0
:100E5C00D293D2AF759F11020F0A207D16C2AF75C7
:100E6C004206D290C291306202D295D2AF759F01E8
:100E7C00020F0AC2AF754206D292C291306202D200
:100E8C0093D2AF759F21020F0A307244207D20C28D
:100E9C00AF754201900146757B01C295D2923062CA
:100EAC0004D293C1B3C290D2AF759F21020F0AC274
:100EBC00AF754201900124757B04C293D2903062CD
:100ECC0005D295020ED4C292D2AF759F01020F0AC1
:100EDC00207D17C2AF75420190011AC29530620293
:100EEC00D293D2AF759F21020F0AC2AF7542019007
:100EFC000106C293306202D295D2AF759F01C265D2
:100F0C0022900104757B00C295C294C293D292D2F6
:100F1C0091D290C26222788076090876090876040C
:100F2C000876FF0876030876FF08760A087601082B
:100F3C007601087601788C76010876FF0876FF0832
:100F4C0076FF0876FF0876FF0876030876FF0876AA
:100F5C00FF0876FF0876250876D0087628087650A4
:100F6C000876040876FF08760208760008767A0878
:100F7C0076FF087601087601087600087603087675
:100F8C0000227887E6FFC2727888E6C39403600873
:100F9C00C27DE630E102D27DC27E7889E630E10284
:100FAC00D27EC3EF94026008758E01D273020FC11A
:100FBC00758E00C273227880E6149000809378A519
:100FCC00F67881E6149000809378A6F67886E6147D
:100FDC0090008D9378A7F67886E6F539C394025085
:100FEC0003753902789CE67538FFB402037538A096
:100FFC00B4030375388278A3E61490009A93F566CF
:10100C00120F0D22227896E6FA7897E6FB7888E69E
:10101C00B40305C3EB940EFB307F047A007BFFC353
:10102C00EB9AFCC3948250027C827572000572ECC0
:10103C008572F0A4C3E5F0947D40F222D27F1111A9
:10104C0012059B12059B7A007B007C10120591E522
:10105C005C2AFA74003BFBDCF37C04C3EB13FBEA65
:0D106C0013FADCF7FEC27F111122757C0023
:10107900757D00E5EF20E6037520000520903FFF10
:10108900E520146006901DFF146000930460037549
:10109900EF1653D9BF7581C043FF8012058C75EFD8
:1010A9000643B203E5B3240220E70DF521E5E32069
:1010B900E0068521B343E301120F0D7580FF75A486
:1010C9000075F19075D47F75908775A5BF75F2BFCE
:1010D90075D50075A60175E241120F0DE4F8F6D831
:1010E900FD756801120F221215D67898867375302E
:1010F90001C2AF1205A51205B512059B1205BC1256
:10110900059B1205C312059BC2AF757C00757D0056
:1011190078FA79FA308707D9FBD8F7021C00120F41
:101129008E120FC21110111178988673120F0D7556
:10113900881075890275C82475910475D84075A8F9
:101149002275B80275E690759B80759D0075D10E64
:1011590075BC5875BB0675BA1175E88012058CD235
:10116900AF12089975360053DACF207E0343DA208F
:10117900307E0343DA1043DA01C2D8C2711205A5E1
:10118900D2617B037A0CE55B70077A0CDB030211F1
:101199001112059B207003021111C270E55CC39402
:1011A9000240E1E52F541F855E5DF55EB55DD5DA38
:1011B900D5C26153DACF207E0343DA20307E034360
:1011C900DA10C2D8C27178A2E67008D274E52F5439
:1011D900E0F52FC2757529001205A0307409C3E521
:1011E90029940A4002D27512059178023074027866
:1011F90000C3E55C9840F0C2AF1205B51205B512FF
:1012090005B5D2AF1205A5754C007888E6B403027E
:101219006106120591788CE6C39401500302130606
:10122900E530C394015003021306757CA5757DF161
:10123900207435C3E55C94FF5003021306C2AF1254
:1012490005CAD2AF1205A0C3E55C940150EFC2AF45
:101259001205B51205961205B5D2AF1205A0C3E560
:101269005C94FF40E902178E7F02D27F11111205AB
:10127900A0C2AFC27F1111AE5CC3E55C947FD2AF4F
:101289005002611612058CC2AF1205CAD2AFDFDA5D
:101299001148C3EE7897F61205A51217117F0AD2E5
:1012A9007F11111205A0C2AFC27F1111AE5CC3E557
:1012B9005C947FD2AF50E612058CC2AF1205B5120D
:1012C90005961205B5D2AFDFD61148EE24037896FC
:1012D900F6F87997E7C394824003985006E8248288
:1012E9007897F61205A51216241217401205A011B7
:1012F90011C3E55C94FF5002413302178E757C00DF
:10130900757D00C3E55C954C4003855C4C1205A0D6
:1013190078017988E7B403027805C3E55C9840024F
:101329004113C2AF1205CA1205CA1205CAD2AF12B9
:1013390005A5753000E4F531F5320531E531F47074
:101349003F0532789AE67819146012783214600DE4
:10135900787D14600878FA146003753200C3E532A9
:1013690098401D120F0D12058C15327531007899B0
:101379008673C2AF1205CAD2AF789886731205A0D8
:10138900120596E52A70053074022111780120743E
:10139900027806C3E55C9840A17888E6C3940360A7
:1013A900031205A0E52A7003021111C2AF120F0D35
:1013B900E4F522F523F524F525F526F567D2AF786E
:1013C90085E6C333F565E4F544F545F546F547F596
:1013D90048F570F52CF52DF53775700875BB1012A9
:1013E900058C12089D30EDFDA8BDA9BEE97001F874
:1013F90088711208A175700875BB10120F8EC2AFE3
:101409007561FF120937852261852262852263D2BF
:10141900AF7522017524017525017526018560695D
:10142900756A017888E6B40307C27D307602D27DF9
:10143900D268D269753300120E66120E95120957D9
:1014490012095E12095712095E120957120BDE12B0
:1014590006AB120CD3120D1A12095E120BCD306EA7
:0D14690003120707206603120853306603C4
:10147600120883120CD3120D4912095E120BDE30CC
:101486006E0312073C120CD3120DC012095E120B2A
:10149600CD306E0312079A120CD3120DEF12095EAD
:1014A600120BDE306E031207F7120CD3120E661201
:1014B600095E12089D120BCD120CD3120E9512085E
:1014C600A112095E3069328564618564628560694E
:1014D600756A0179187A0CC3E53399400FC269D24F
:1014E6006A8A358564618564630214FFC3E55C948A
:1014F60001400302145502158D306A25206C22E541
:1015060035147006C26AD26B8155F535C3E55C9415
:101516000140030214557888E6C39403600302155C
:101526008D75360078FA79A4E760027803C3E55F23
:10153600985054307404E52A604D7888E6B4031751
:10154600207D05207607A15D307602A15D206C071F
:10155600D26C856461819478F0306C05856461781D
:1015660020C3E5419850028155306C1BC26CC27D88
:10157600307602D27DD26A75351285646181550551
:1015860036E55C6002A190753600C2AF120F0D7889
:1015960087E6FE7602120F8E7887EEF6E4F522F5E0
:1015A60023F524F525F526F565752C00752D00D255
:1015B600AF1205A0120F0D78A4E66006C292C29182
:1015C600C290307409C3E536940440022111613E8D
:1015D600901A0D7820121666E520B4550CA3121643
:1015E60066E520B4AA03021604757CA5757DF11282
:1015F6000F22121624757C00757D00021623901AA0
:101606000378807B0A121666A308DBF9901A0F7816
:101616008C7B19121666A308DBF9901A2822C2AF32
:101626001216A9121686901A00740E12166BA3745F
:101636000912166BA3741512166B901A0378807B29
:101646000A12166AA308DBF9901A0F788C7B191216
:10165600166AA308DBF91216BC12169A901A2822EB
:10166600E493F622E6438F01538FFDFFC3E583948F
:101676001C400122EF857CB7857DB7F0538FFE2293
:10168600438F02438F01857CB7857DB7901A0DF095
:10169600538FFC22901A0D7455D16B901A0E74AAB2
:1016A600D16B227A3079D07820901A40D166E52025
:1016B600F709A3DAF7227A3079D0901A40E7D16B8E
:1016C60009A3DAF922AB74A875BB01027980BB02C3
:1016D600027981BB03027982BB04027984BB0502CD
:1016E6007986BB06027992BB07027987BB08027925
:1016F600A3BB0902799CBB0A027988BB0B027989D4
:10170600E8F7227C051205A5DCFB22C2AF1205B55F
:101716001205BC1205C31205CA1205961205B512AA
:1017260005BC1205C31205CA1205961205B51205A7
:10173600BC1205C31205CAD2AF22C2AF1205CA1225
:1017460005C31205BC1205B51205961205CA120587
:10175600C31205BC1205B51205961205CA1205C3B9
:101766001205BC1205B5D2AF22AE74AF75C2AF1268
:1017760005B51205B51205B5120596DEF21205CAB3
:10178600120596DFF8D2AF22F111F109F10975744D
:1017960001757501757600F16F7C05AD5C1205A5C6
:1017A600C3ED955C70F5C3E55C9401400AC3E55C46
:1017B60094FF40320217CAD1CBD124F111C2AF75C2
:1017C600EF16F109DCD50576C3E576940350028061
:1017D600C6F1090575E5741490009F93F808C3E5F2
:1017E6007598500280AEF109F1090574C3E5749449
:1017F6000C5002809C120F22121624C2AF75EF16EF
:03180600121709AD
:0319FD000210765F
:101A00000E0915090904FF03FF0A01010155AA0186
:101A1000FFFFFFFFFF03FFFFFF25D0285004FF0259
:091A2000007AFF0101000300FF40
:101A400023585031384123202020202020202020DE
:101A500023424C48454C4923463333302320202031
:101A60002020202020202020202020202020202076
:101C0000C2AFC2D353D9BF7581C043B20343FF8073
:101C1000752438752503B1DC7529A5752AF175E29F
:101C20004043F18053A47F75D4FFD2877DFA7803B7
:101C300079E67C10752200752300901DE97B0675FE
:101C400024987525013087028145208708D8FBD963
:101C5000F9DCF781B7308708D8FBD9F9DCF781B711
:101C6000B19CE493A3C39A6004DDC381B7DBDBB10D
:101C70008E6002812E7B08E493FAA3B16FDBF87AC1
:101C800030B16F752200752300B18EEAFCEBFDC305
:101C9000ED94FE400EB18E8A278B28ED30E0048A49
:101CA000828B83B18E7AC270D8C3ED94FE601950D6
:101CB000CEBD002BEC600F7520007521FF7529004B
:101CC000752A000200008100A827A9280809D80465
:101CD000D90281DCB192EA89AAF281CE0D81A3C337
:101CE000ED94035053EDA2E092007AC5C3E58294CF
:101CF00000E583941C508A200010438F02438F011B
:101D00008529B7852AB7F0300029A827A92808090E
:101D1000438F01538FFDD804D902A133C3E58394C7
:101D20001C4003A3A11689AAE28529B7852AB7F02A
:101D3000A3A116538FFC817F7AC1BD030CE493A34A
:101D4000FAB153DCF8B14B817F8181AA22AB23B178
:101D50006FEBFAEA6222752608C3E52313F523E543
:101D60002213F52250066323A0632201D526EAB18F
:101D7000DCB1DC75260AEAF4200102D287300102C8
:101D8000C287B1DCC3134002C201D526EB22B19257
:101D9000EAFB208702A192308702A197752608AE40
:101DA00024AF25C3EF13FFEE13FEB1E0B1DCC3EAAD
:101DB000133087024480FA30E703632201C3E5232E
:101DC00013F523E52213F52250066323A0632201B5
:101DD000D526D9E52265236523F52222AE24AF2539
:101DE0000E0FDEFEDFFCD20122424C48656C6934E6
:071DF000373164F3300601F6
:00000001FF
